:020000020000FC
:1000000055CDA5C1000000001FC0000093C0000036
:1000100000009DC000000000000000000203040674
:10002000080C10182030406080000406080C1018DE
:100030002030406080A0C00000070F1F3F00050572
:100040000D050305030302004FB662FD0EC05520E7
:1000500009F00994C52DC095089483FDC795C4BDCA
:10006000C093A10064604FBE1895C09164000894CD
:1000700083FDC795C4BDC093A1006B7FC091640090
:10008000CF3F09F420C070FF02C082FD05C04FBE03
:10009000919890989398189575FD0EC065FD0CC0C9
:1000A000C091B300C0FD9498C1FD9798C2FD95988A
:1000B000CAEFC095CA95F1F79198909893982092BD
:1000C000A1004FBE189524BCCC27C064C8BF646093
:1000D000F6CFC0CF70FFBECF65FDBCCF919ABACF2F
:1000E00070FFB8CF65FDB6CF909AB4CF70FFB2CF96
:1000F00065FDB0CF939AAECF949A70FFABCF65FDFC
:10010000A9CFC7E0CA95F1F7919AA4CF979A70FF4B
:10011000A1CF65FD9FCFC7E0CA95F1F7909A9ACF1E
:10012000959A70FF97CF65FD95CFC7E0CA95F1F717
:10013000939A90CF4FB6C9B7CF7EC9BF6E7FCCB56B
:10014000CE0DDDB5DF1DDBBDCABD4FBE18953FB678
:100150008F7EABB7A074A2118061A0E0ABBFA9B73E
:10016000AE7FA9BF7894A0916800AA2341F085FDD5
:100170002AC0A0916800AA95A093680024C040E01E
:1001800050E085FD14C0A0B396FDA095A2FD4FEFF1
:10019000A3E096FDA2E0A5BFAA27A064AABF8D7F19
:1001A000A0B396FDA095A2FD5FEF451741F7A8E12A
:1001B00061FDA093680085FD03C0A8E1A0936800DD
:1001C00040939700816085FD0EC0A0916900AA232D
:1001D00031F0A0916900AA95A093690004C08061E4
:1001E000AA27A064AABF80FF38C0A09197004A2F19
:1001F00061FF8E7F85FD18C0403F08F040EFA42FBF
:10020000A295AF704A0F5091B800533069F0A6958F
:10021000A69550FD01C0A69552FD03C0A41B4A2F10
:1002200003C04A0F08F44FEFA091A0004A1708F44A
:100230004A2F40936100A72FA67079F0A0916D001E
:10024000A695A69556E0A50F50916100A50FA09325
:10025000610018F4AFEFA0936100A0916100A0933A
:10026000630040916300A0919C004A1708F04A2F58
:10027000542EA091A200AA2309F422C0542F5A1B85
:1002800010F4A42F50E0BA2E8894AA1FAA2EA09191
:10029000A400A095AA22A50E58F0A091A300A21533
:1002A00009F0AA95AA0EA093A30048F04A2D08C011
:1002B000A091A300BA1608F0A395A093A3004FEF56
:1002C000409364007F7D485F08F07062A52DA034E4
:1002D00008F06860A0916000A395A093600051F0C1
:1002E000F894A9B7A160A9BF84FF02C0A0E4ABBF86
:1002F0003FBE1895A0917400A395A093740041E0AF
:1003000050916800552329F085FF03C05A955093FA
:100310006800A0919700A13018F020929A000DC0BB
:1003200020929B002092A500A0919A00AF5FA0931D
:100330009A0018F0AFEFA0939A00F894A9B7A160C3
:10034000A9BF84FF02C0A0E4ABBF3FBE18953FB673
:100350004CB55DB58F7EABB7A074A2118061A0E0F3
:10036000ABBFA9B7AE7FA9BF789481FD23C0A2E03F
:1003700096FDA3E0A5BF8260A0B396FDA095A2FF65
:1003800005C040936500509366003EC1A3E096FD12
:10039000A2E0A5BFAA27A064AABF8D7F85FF01C0E8
:1003A00026C140E0A0B396FDA095A2FD20C14093D8
:1003B00097000FC1A3E096FDA2E0A5BF8D7F61FF6E
:1003C00071C0A2E096FDA3E0A5BFAA27A064AABFC2
:1003D00082604093920050939300A09090004A193D
:1003E000B09091005B09BB24A22C4C38520518F444
:1003F0002092960049C0A091D600AA2359F1483C0A
:10040000520528F4A0E1BA2EAAE0AA2E23C048364D
:10041000A1E05A0728F4A8E0BA2EAFE0AA2E1AC02D
:10042000403DA2E05A0728F4A4E0BA2EAEE1AA2E7D
:1004300011C0403AA5E05A0728F4A2E0BA2EACE376
:10044000AA2E08C04839A8E05A0720F4A1E0BA2E25
:10045000A8E7AA2EC42EA0919400CA1AD52EA09166
:100460009500DA0ADD202AF4AFEFC094D094CA1ABE
:10047000DA0A20929600A8E0A210A0E0CA14DA06D8
:1004800018F4A1E0A0939600409394005093950037
:1004900040919200509193004093900050939100AE
:1004A00002E097C0A09165004A1BA09166005A0B1C
:1004B00094FD82C093FD80C092FD7CC086FF03C086
:1004C000D52EC42E0CC05695479591FD73C05695F8
:1004D000479590FD6FC0D52EC42ED694C79461FD6C
:1004E00019C0AC2DAC51AD2DA24008F005C0DD20E7
:1004F00089F4AC2DA85C70F4A0916700A395AA23A1
:1005000011F0A0936700AA3008F471C02092970000
:1005100081606DC0A0916700AA2319F0AA95A093ED
:100520006700A22C5091BC0097FD06C0A090CA00A5
:10053000533011F4A090D200AAEFAA0EA22DA21D52
:10054000CA18DA0A4FB74170533049F4442321F0F6
:1005500087FD05C0806803C087FF01C08F774423F3
:1005600059F0533031F4AFEFC094D094CA1ADA0A7C
:1005700003C040E050E020C0533049F4CC0CDD1CF7
:10058000AAE0CA1AD20818F4A0E0CA2ED22CAFEF03
:10059000CA16D20418F04FEF50E00EC0A091AE0082
:1005A000CA9E412D000C441F50E008F012C04FEFCE
:1005B00050E00FC05695479594FF07C0552309F0AA
:1005C0004FEFA42FA6954A0F521D4F3F520508F03A
:1005D0004FEF40939700816061FF09C0AFE1A095A4
:1005E000A923AB299A2F8F7DBB2009F48062A8E153
:1005F000A093680085FF03C0AAE0A093680061FD96
:1006000003C085FD01C08F7E85FD03C0A6E0A093D9
:100610006900F894A9B7A160A9BF84FF02C0A0E453
:10062000ABBF3FBE189511E00AC013E008C01AE046
:1006300006C01EE104C014E602C018EC00C005E1CB
:10064000BB27BA95F1F70A95D9F71A95C1F708951E
:100650002AE338E709C020E33CE806C02AE234EB8D
:1006600003C025E238EC00C012E095FD9F7D95FFA8
:100670009062BB27979ABA95F1F7909ABA95F1F7DD
:100680009098BA95F1F79798BA95F1F7919AB09139
:10069000AF00BA95F1F79198B7E8BA95F1F71A95C6
:1006A00021F7022FB22FBA95F1F70A95D9F73A95AB
:1006B000D9F6979A0895221B39E0001F3A9509F45C
:1006C0000895221F211B18F4210F8894F6CF089457
:1006D000F4CF622C722CB0E08894B395221F331FA4
:1006E000E0F7379527958894912E802E020B130BF7
:1006F00010F4192D082D10F4889401C00894661C7C
:10070000771CBA9571F7172D062D0895322D1123F8
:100710002AF43A9500951095031B130BF894029F49
:10072000712C002D129F912C802C7894780C172D11
:10073000921C292DB4E06B2E2695179507956A9487
:10074000D9F7332321F000951095031B130B08955F
:10075000089510917B00169500917A000795B0914D
:100760007F00B01B0B2FB0918000B10B1B2F28F422
:100770000038BFEF1B0740F009C00F37120508F41F
:1007800005C00FE710E002C000E81FEF00938400EF
:1007900010938500089500918400B09181000B0FA3
:1007A00010918500B09182001B1F20E030918500E0
:1007B00033230AF42A95B09183002B1F1AF4203FAB
:1007C00040F00AC02F3008F407C00FEF1FEF2FE0F2
:1007D00003C000E010E020EF30916300B0919C0076
:1007E0003B1718F4323030F009C0B0918500BB23BC
:1007F0005AF004C0B0918500BB2332F4009381000D
:10080000109382002093830008952091D8000091D6
:100810008400000F10918500111F78DF11232AF446
:100820000038BFEF1B0740F009C00F37120508F46E
:1008300005C00FE710E002C000E81FEF002352F0F0
:10084000B0916200B01B0B2F18F0013008F00AC005
:1008500001E008C000950F5FB09162000B0F08F037
:1008600001C00FEF0093860008952091D9000091F8
:100870008200109183004ADF11232AF40130BFEF78
:100880001B0740F009C00F3F120508F405C00FEF29
:1008900010E002C001E01FEF112352F0B09186007A
:1008A000B01B0B2F18F0013008F00AC001E008C09F
:1008B00000950F5FB09186000B0F08F001C00FEF9D
:1008C0000093630008950FEF677F71FD29C072FDEB
:1008D00009C06860B0917B00BA3020F0B52DB0340B
:1008E00008F4677FB091D500BB23D1F0B0917B00B5
:1008F000BB23B1F00FEF10917B00DDDEF894B091D7
:10090000730072FDB5E00B9F112D002D789411231B
:1009100009F00FEFB0919F000B1710F400919F00AA
:1009200000939E00089500917A0010917B0000547E
:100930001140B0919E0010F4BA9501C0B39511F02A
:10094000B0939E00089500C008952091B700B6B1FD
:10095000B6FDFBCF04B115B1B6B1BF77B6B9B09152
:10096000AC00B395B093AC00B83060F12092AC000D
:10097000B091D400BB2321F1112329F0B091AD0037
:10098000BF3F61F009C0B091AD000B1739F020F402
:10099000BB2321F0BA9502C0B395E1F300919C000E
:1009A000B093AD00B03050F400ECB03038F400E853
:1009B000B03020F400E4B03008F400E000939C0074
:1009C000777F0895B0919C00B39511F0B0939C008F
:1009D000B091AC00B73009F47860089502E3F89460
:1009E000B091DA000B9F012D000C001F7894B0919C
:1009F0009C000B1710F000919C0000936100009385
:100A00006300502E0093640000939F00089520928D
:100A10007A00B0EFB0937B000895F8940CB51DB543
:100A20002091740078943091750060907600009366
:100A3000750010937600031B160971FD03C076FD47
:100A400081C02BC070907700209377002709222364
:100A500011F00FEF1FEF80907800909079003093A5
:100A60007800609279006918161910937C00009143
:100A70007500109176000819190920917A003091BB
:100A80007B0036952795020F131F10F40FEF1FEF11
:100A900000937A0010937B0029C020917A00309156
:100AA0007B003901B4E08B2EB2E09B2E343010F085
:100AB0008A949A94383010F08A949A947694679431
:100AC0008A94E1F726193709992021F016950795A0
:100AD0009A94E1F7200F311F20937A0030937B0026
:100AE00028F43FEF30937A0030937B00323008F4E3
:100AF000706471FF02C0B3E00DC0B091C6000091F8
:100B00007100023838F0B395003A08F0B395B6306A
:100B100008F0B5E09B2EB4E08B2E10917B00009185
:100B20007A0024E0169507952A95E1F7081912092D
:100B300028F0B02FB250B12FB20910F402E010E04B
:100B4000980126C020917A0030917B00390176947B
:100B500067946694669466942619320906950695FC
:100B6000200F321D20937A0030937B00323008F042
:100B70007F7B04E036952795369527952695269513
:100B8000201B10F0223008F422E089019090C6006A
:100B900060FDFECFE0908C00F0908D006160B9B7F1
:100BA000B061B9BF380176FD44C076946794009374
:100BB0008C0010938D00B92DB330E1F0B0FD04C06E
:100BC000060D171D930106C0000F111F02501209D8
:100BD00022E030E0B92DB33068F020938E003093DE
:100BE0008F00009388001093890060928A007092B1
:100BF0008B003DC000938E0010938F0020938800DF
:100C00003093890060928A0070928B0071FF10C04F
:100C1000B0916D00B33060F000918F0010917C00B6
:100C20001595010F28F022F020928E0000938F007E
:100C30001EC0669400938C00B92DB33091F0B0FDC6
:100C400003C0060D262D03C0000F025022E0B92D6F
:100C5000B33038F020938E000093880060928A00B1
:100C600006C000938E002093880060928A00009155
:100C70007D0002FD0350013031F495FD0CC0B2E05F
:100C8000B06CB7B90BC0023021F4B3E0B06CB7B9A7
:100C900005C095FDF4CFB4E0B06CB7B90091A400E5
:100CA000000F10F4BBE60B270093A40060FDFECFFD
:100CB000B2E0B0936E006160B9B7B061B9BFB72F51
:100CC000B670A1F020917A0030917B00369527957F
:100CD000F8940CB51DB5020F131F1BBD0ABD616052
:100CE000B0E1B8BFB9B7B061B9BF78940895606199
:100CF00020927E0020E067FD20E206C06061209225
:100D00007E0020E267FD20E0789401E076FD11C0CE
:100D1000B72FB67009F06F7EB0917B00B55048F0E8
:100D200002E0B55020F003E0B55008F006E071FD98
:100D30000AE060FD12C0B0917E00BB2371F071FF2C
:100D400008C0B0916D00B33020F0B0916E00BA953C
:100D500019F4789470615CC0AEDF789400000000F4
:100D6000F89476FD16C010917B00173008F017E05C
:100D7000B5E01B0F72FD10E183FF110F62FF110F31
:100D800071FD12E8B4B56090A100B61990F2B10BF4
:100D900080F2B0B7B77FB0BFB8B1B0B7B860B0BF7E
:100DA000B0917E00B395B0937E00B8B176FD06C0D9
:100DB000B1E071FDB2E0BA95F1F7B8B1B072B21717
:100DC00009F01BC071FF05C003950A3008F00395B8
:100DD000B0CF64FF99CF6F7E3CB56DB470907A0050
:100DE00080907B00370D681C6BBC3ABD6160B0E140
:100DF000B8BFB9B7B061B9BF87CFB0916D00B2309D
:100E000008F482CF64FD80CF0A9509F092CF7F7EEF
:100E100020918E0030918F00F894B0E1B8BF0CB5EE
:100E20001DB5020F131F1BBD0ABDE0908800F09096
:100E300089006160B9B7B061B9BF7894B72FB67057
:100E400039F0B0916D0072FFB395B0936D0009C099
:100E500074FF07C067FD05C064FD03C0BF91BF916B
:100E6000E1C4089500E063FF03C064FF01C001E036
:100E7000F89410917100B7E01B9F212D102D7894EC
:100E8000200F26951795269517952695179510935B
:100E90007100183718F4B8E7B09371000091710031
:100EA000B09172000B1720F060629198909893981F
:100EB00060FDFECFE0908A00F0908B006160B9B7D2
:100EC000B061B9BF0895B2E095FD07C0F894B09342
:100ED0007D00979A94987894E5C0F894B0937D003B
:100EE000979A95987894DEC0B3E082FF24C095FD70
:100EF00011C002E0F894B0937D00E6E8F0E00093C2
:100F0000B3009398959A62FF02C0909A01C0979897
:100F10007894C8C002E0F894B0937D00E6E8F0E071
:100F20000093B3009198949A62FF02C0909A01C016
:100F300097987894B7C095FD0BC0F894B0937D0056
:100F4000E0E7F0E0939862FF01C0909A7894AAC01D
:100F5000F894B0937D00E0E7F0E0919862FF01C063
:100F6000909A78949FC0B4E095FD07C0F894B09330
:100F70007D00949A9598789495C0F894B0937D00EC
:100F8000959A949878948EC0B5E082FF24C095FD20
:100F900011C001E0F894B0937D00ECE7F0E000931D
:100FA000B3009098979A62FF02C0919A01C09498FA
:100FB000789478C004E0F894B0937D00E0E9F0E024
:100FC0000093B3009098979A62FF02C0939A01C071
:100FD0009598789467C095FD0BC0F894B0937D0008
:100FE000EAE6F0E0909862FF01C0919A78945AC0C6
:100FF000F894B0937D00E6E7F0E0909862FF01C0BE
:10100000939A78944FC0B6E095FD07C0F894B093DA
:101010007D00959A9798789445C0F894B0937D0098
:10102000949A979878943EC0B1E082FF24C095FDD1
:1010300011C004E0F894B0937D00E0E9F0E0009383
:10104000B3009198949A62FF02C0939A01C0959858
:10105000789428C001E0F894B0937D00ECE7F0E0CC
:101060000093B3009398959A62FF02C0919A01C0D1
:101070009498789417C095FD0BC0F894B0937D00B8
:10108000E6E7F0E0919862FF01C0939A78940AC075
:10109000F894B0937D00EAE6F0E0939862FF01C017
:1010A000919A78946F7D089529E630E0F9012092B5
:1010B000B300919890989398949A979A959A6B7F89
:1010C0000895A4EBB0E00FEF0D930D930D930D93E6
:1010D00003E00D9304E00D9309E00D9303E00D93FD
:1010E00001E00D9301E00D93A0ECB0E001E00D9361
:1010F0000FEF0D930D930D930D930D9303E00D934F
:101100000FEF0D930FEF0D930D9305E20D9300ED8F
:101110000D930AEF0D930AEF0D9304E00D930FEF7B
:101120000D9301E00D9300E00D930AE70D930FEF8F
:101130000D9300E00D9301E00D9300E00D9303E0AB
:101140000D9308952091BB008B7F233009F48460B8
:10115000B091BC00B33019F09F7DB1FD90629F7BD0
:10116000B091BD00B1FD9064223011F0886001C0E3
:10117000877F08950A95E00FF21DB4910895ECE180
:10118000F0E00091B400F6DFB093D800ECE1F0E0BD
:101190000091B500EFDFB093D900EAE2F0E00091F2
:1011A000BA00E8DFB093DA00B091D0000FEF1CE096
:1011B000B23011F400EA1AE0B33011F402E815E09D
:1011C0000093720010937300E8E3F0E00091D70001
:1011D000D1DFB093A200089508952091CA00309104
:1011E000CB00B091BC00B33009F43E5097FF02C071
:1011F00020E03FEFB32FB21B6B2EB25810F4B2E8D1
:101200006B2E00E00395609EB12DBD57D8F300937F
:10121000AE0008959068E1DF0CDA20E030E0B0E144
:101220006B2E03DAB09197002B0F321D6A94C9F729
:10123000B4E036952795BA95E1F7822E9F77CDDFFA
:101240000895F894E3E0F0E0B9E0B7BFB491B07866
:10125000C1F3F894A895B1B5B861B1BDB0E0B1BD26
:10126000B4E0BEBFBFE5BDBF1FDFB0E0B8BBB0E1BB
:10127000B7BBB0E0B5BBB0E0B4BBB0EBB2BBBBEB4F
:10128000B1BB2224A0E0B0E02D92AA31E9F7A0E69C
:10129000B0E00FEF2D920A95E9F7B1E0B093A4000A
:1012A00010DFF4D2B7E0B06CB7B9B6B1B460B068D3
:1012B000B6B90091CC000093AF00B1E0B0936A00E2
:1012C000F894BBD9C5D9B5D9C6D9B3D9C7D9B1D97D
:1012D00064D3B3D9B2D9AFD9F8940AEF1AEFA0B357
:1012E00096FDA095A2FF1FC01A95C9F70A95B1F700
:1012F000E0E0FCE1B591B43E39F4B591B03E21F4A3
:10130000B591BF3F09F40CC0E0E0F395F395B591BA
:10131000B83F49F4B591B43931F4B591BA3A19F4FA
:10132000EE27F69509940EDF2ADF56DF56DF00918F
:10133000CC000093AF00B8DEB2E0B3BFB2E0BEBDF8
:10134000B2E0B5BDB1E5B8BFB9BFB0B7B77FB0BF08
:10135000B8B1B0B7B860B0BF66D97894F4DAB3E08A
:1013600096FDB2E0B5BFB0E4BBBFBB27B064BABF67
:101370008D7F63D9626033E02CE0B0919600BB238F
:1013800021F42CE03A9509F4A7CF53D980FFA4CFDC
:101390008E7FB0919700B23078F3B92FBF71009172
:1013A000990000939800B0939900B01729F72A95F7
:1013B00021F76D7FB3E096FDB2E0B5BFBB27B06407
:1013C000BABF8D7FB091D600BB2321F48062B92FC4
:1013D000B0709B2F8F7B209267002DD985FF05C0B1
:1013E000B0916700BA3008F080641FD902E085FF31
:1013F00001C000E0B0919700B017B8F3F89428D975
:1014000027D926D9789419D920928700B091BC00A9
:10141000B33009F474C009D9B091C000B13008F4F8
:101420006EC0B0916A00B13008F469C085FD18C083
:10143000B0919700BF3F08F462C0F89412D9789435
:10144000FAD8B0919700B130C0F7F89401D9EFD82D
:10145000FFD87894F0D8B0919700BF3FB0F3CFC2D7
:10146000B8E09B2E9068F894B8DE7894E4D8F894AD
:101470009F77B3DE80909700B0919700BF37789444
:1014800008F445C0D0D8F894ECD878949A9451F7E1
:10149000C1DEB82DB550B093CB00CFD8F89423D28D
:1014A00081D27894BAE09B2E9068F89496DE789476
:1014B000C2D8F8949F7791DE80909700B091970002
:1014C000BF37789478F7AFD8F894C2D8B0D8C0D8DE
:1014D00078949A9449F79EDEB82DBB5FB093CA000A
:1014E000ACD8F89400D26DD27894A5D8F89475DE73
:1014F0007894B0919700BF3F08F498CF80C20091D4
:101500009700B09187000B1710F00093870093D8D5
:1015100001E0B091BC00B35009F405E0B091970030
:10152000B01708F073CFF8949CD89BD89AD87894C9
:1015300084D820926A0020926B0020926C00B091B7
:101540006B00B395B0936B00BF3F69F5B0916C0031
:10155000B395B0936C00B091CE0009E1BA9559F003
:1015600002E3BA9541F00DE7BA9529F00AEFBA9572
:1015700011F020926C00B0916C00B017A0F0B09107
:101580006C00BA95B0936C00B4EBB0936B00B09163
:10159000CD00B093AF00F89464D87894B091CC00AB
:1015A000B093AF0048D843D8B0916800BB2319F47A
:1015B00085FF01C091CE01E085FD01C006E0B0913C
:1015C0009700B01708F4BBCFB091BC00B35009F03E
:1015D00032D8B0916800BB2309F47ECEF89464DD64
:1015E000209261002092620020926300522C20928F
:1015F00064002092A3007894B091B900BB0FB0931F
:10160000A00020927F0020928000209281002092F2
:101610008200209283002092AC0060E070E0209273
:101620007100B8E0B093AC007860FDD7B7E073FD0F
:10163000B7E0B06CB7B9B6B1B068B064B6B9B6B11E
:10164000B6FDFDCF04B115B1B6B1BF77B6B9112360
:1016500009F00FEF0093AD0078D9B8E0B093AC007B
:1016600078608090BB00B2E0B093BB006BDD8092ED
:10167000BB00F894BFEFB0939C00B0D9B09161006B
:10168000B0939C00B0939D00B0939E007894B1E01D
:10169000B0936100B09363005B2EB0936400B0938D
:1016A000A600B0919B00B093A500B091BC00B330F0
:1016B00019F49F7D87FD90627160726020926D00C9
:1016C000A2DCB2DCA4D9A9D9A2D9A7D9A0D906C0D5
:1016D000F89438DD78942092AC00777F0FDB38D80F
:1016E000C1DBF1DB9AD903DB66FD33D876FFEBD89B
:1016F00076FD19D9B7DBF8DB90D900DB66FD4BD856
:10170000B1DB31DC8AD9F3DA66FD7FD8ABDB3CDCB8
:1017100084D9F4DA66FDA9D8A5DB75DC7ED9E7DAD1
:10172000B7E073FDB7E0B06CB7B9B6B1B068B064FC
:10173000B6B998DB79DC71D908D971FF23C067FD90
:1017400021C0B0919F00B0939C00B0939D00B091D8
:101750009B00B093A500B1E0B093A60018E12CE087
:10176000B0916D00B11740F07D7F746020936F00E1
:10177000BFEFB0939C0006C0B0919700B13008F065
:10178000ADCF5AC072FF10C067FD0EC0B0916F00A0
:10179000BA9511F47B7F9CCFB0936F00B091970006
:1017A000B13008F09BCF48C020927000B0919A00F1
:1017B00002E8B01708F040C085FF04C0B09168008F
:1017C000BB23D1F1B091BC00B33081F495FD03C0CF
:1017D00087FD04C00BC087FF01C008C067FD06C0BD
:1017E0006068B0919F00B0939C008DCF00EF67FFC1
:1017F00005C0B0919F00B0939C0000E2B0917B00C7
:10180000B01708F46BCF67FF17C06F779F7D87FD18
:1018100090627460B2E1B0936F00B0919F00B0939A
:101820009C005CCFB0917000B395B0937000B09104
:101830009700BB2309F002C020927000F89434DCBA
:101840008090BB00B2E0B093BB007CDC8092BB0018
:10185000209261002092620020926300522C20921C
:1018600064002092A0007E7F7894DDD61DDCB7E076
:10187000B06CB7B9B6B1B460B068B6B985FF05C091
:10188000B0917000B53008F027CD55CEEDE0F0E016
:1018900023D00A3509F01BC0EEE0F0E01DD0053A78
:1018A00009F015C03AE0A4EBB0E0E3E0F0E014D0BA
:1018B0000D9331963A95D9F738E1A0ECB0E0EFE01E
:1018C000F0E00AD00D9331963A95D9F702C0F9DBD2
:1018D0000AD0E7E2F0E00895E199FECFEEBBFFBB4E
:1018E000E09A0DB308951ED03AE0A4EBB0E0E3E037
:1018F000F0E00D910FD031963A95D9F738E1A0EC90
:10190000B0E0EFE0F0E00D9105D031963A95D9F7CF
:1019100012D00895E199FECF0DBBEEBBFFBBE29A5A
:10192000E19A0895EDE0F0E00FEFF4DFEEE0F0E093
:101930000FEFF0DF0895EDE0F0E00AE5EBDFEEE019
:10194000F0E005EAE7DF08953091B0000091B100C2
:10195000313011F40093B800323011F40093B90023
:10196000333011F40093BA00343011F40093C60000
:10197000353011F40093BB00363011F40093D700DA
:10198000373011F40093D000383011F40093BC00CC
:10199000393011F40093BD00089525E04ED62A9504
:1019A000E9F7089555D657D659D65BD640D650D6C6
:1019B00052D654D656D63BD64BD64DD64FD651D608
:1019C00008954FD64BD647D643D631D64AD646D6BB
:1019D00042D63ED62CD645D641D63DD639D60895E8
:1019E0008090B0009090B10033D632D631D61FD659
:1019F0008A94D1F736D61BD69A94E1F70895F894D5
:101A0000D1DF7894CADFC9DFB1E0B093B000B1E0B4
:101A1000B093B1002092B200F894E2DF7894B5E080
:101A20006B2E7090970009D6B09197007B16C9F77E
:101A3000B13018F0BF3F40F107C086DFF89453DFA4
:101A4000B1DFB8E0B1BDA9DF6A9459F7B091B20037
:101A5000B395B093B200B33008F4DECF9EDFB091FF
:101A6000B100B395B093B100F894B091B000BA95BD
:101A7000EEE3F0E0EB0FF21D049178940395B09142
:101A8000B100B01708F4C6CF88DF87DFB091B0008F
:101A9000B395B093B000B091B000BA3008F4B7CFAE
:0E1AA00010DBF89420DFB8E0B1BD77DFCACBD1
:00000001FF
